:020000040000FA
:020000000E28C8
:10000800FE00030EF0000A08F100831203137F08B4
:10001800F20013280F28F301F40183013B280B1D7C
:1000280030280130F3070318F40A0030F407740885
:10003800803AFF008F307F02031D2428FF307302AF
:10004800031C2F28F301F40183120313861D2E28A5
:1000580086112F2886150B11720883120313FF00CF
:1000680071088A00700E8300FE0E7E0E090083164A
:1000780003138611811281150114811401158B1641
:040088008B17452865
:02400E006DFF44
:00000001FF
